:100000000C941E060C9469280C9496280C944606B1
:100010000C9446060C94E9120C9446060C94460681
:100020000C9446060C9446060C9446060C94460620
:100030000C9446060C9446060C9446060C94460610
:100040000C94C3280C9446060C94B12C0C94F42CFC
:100050000C9446060C9446060C9446060C944606F0
:100060000C9446060C944606D0183219111914192E
:1000700017191A191D192019231932192C19641A64
:10008000661A661A641A661A661A661A661A661A72
:10009000661A661A661A661A661A661A661A661A60
:1000A000EA19661A661A661A661A661A5B19661AD9
:1000B000661A661A661A661A661A661A661A661A40
:1000C000661A661A661A661A661A661AF619F61912
:1000D000F619F619F619F619F619F619F619661A37
:1000E000661A661A661A661A661A5B19F519F51900
:1000F000F519F519661A031A091A0F1A151A1B1A97
:10010000211A271A2D1A371A411A4B1A551A9C19F7
:100110005E19661A661A661A661AEA19661A661A65
:10012000661A661A661A661A661A661AF419F419B5
:10013000F419F419661A031A091A0F1A151A1B1A58
:10014000211A271A2D1A371A411A4B1A551A9C19B7
:100150005E19661A661A661A661AEA19991A991ABF
:10016000991A991A991A991A991A991A991A991AF7
:10017000991A991A991AAF1BAF1BAF1BAF1BAF1B74
:10018000AF1BDE1AE81AF21AFC1A591B631B721B0A
:10019000831B0B1D201D2C1D351D441D691D721D4B
:1001A000BB1D841DCE20D420DA20E120EF201121B8
:1001B0002F21456E746572206D656E752E2E2E0092
:1001C000546F67676C6564206D6963726F50504D42
:1001D00000546F67676C656420696E76657274653C
:1001E000642050504D2100546F67676C6564205443
:1001F00058206D7574696E672100546F67676C6570
:10020000642074656C656D65747279210050726F3D
:10021000746F636F6C206572726F72207769746897
:100220002052580054696D656F7574207768656E4B
:1002300020636F6E6E656374696E6720746F205201
:100240005800507265737320616E79206B65792058
:10025000746F2063616E63656C00436F6E6E6563DF
:1002600074696E6720746F2052582C20706F776508
:100270007220757020746865205258202877697440
:10028000682062696E6420706C7567206966206EF4
:100290006F74207573696E6720616C776179732064
:1002A00062696E642900546F67676C656420276912
:1002B0006D6D656469617465206F75747075742700
:1002C00000546F67676C65642027736C61766520E6
:1002D0006D6F64652700546F67676C6564202761E4
:1002E0006C776179732062696E642700546F676769
:1002F0006C65642050504D206368616E6E656C20A3
:100300006C696D69740053657420525353492069B8
:100310006E6A656374696F6E206368616E6E656C8A
:100320002028303D3D64697361626C652900536526
:10033000742050504D206D696E696D756D20737914
:100340006E630053657420626561636F6E20696E31
:1003500074657276616C0053657420626561636FC9
:100360006E2064656C617900536574206265616319
:100370006F6E206672657175656E637920696E2097
:10038000487A3A20303D64697361626C652C205074
:10039000783D504D52206368616E6E656C20782CFC
:1003A0002046783D465253206368616E6E656C202E
:1003B00078005365742050574D2073746F7020641B
:1003C000656C61792028302064697361626C6564B2
:1003D0002C20312D323535203D3D20302E317320FB
:1003E0002D2035306D696E29005365742050504DB5
:1003F0002073746F702064656C61792028302064EC
:10040000697361626C65642C20312D323535203D75
:100410003D20302E3173202D2035306D696E29003E
:10042000536574206661696C736166652064656CF0
:1004300061792028302064697361626C65642C20C6
:10044000312D323535203D3D20302E3173202D2089
:1004500035306D696E29002A2A2A2A2A2A2A2A2A50
:100460002A2A2A2A2A2A2A2A2A2A2A2A2A2A2A2AEC
:100470002A2A2A2A0052582041636B6564202D20C5
:1004800072657665727420737563636573736675E0
:100490006C21002A2A2A2A2A2A2A2A2A2A2A2A2AAD
:1004A0002A2A2A2A2A2A2A2A2A2A2A2A2A2A2A2AAC
:1004B000002A2A2A2A2A2A2A2A2A2A2A2A2A2A2AC6
:1004C0002A2A2A2A2A2A2A2A2A2A2A2A2A2A00528E
:1004D000582041636B6564202D20757064617465DC
:1004E000207375636365737366756C21002A2A2A0D
:1004F0002A2A2A2A2A2A2A2A2A2A2A2A2A2A2A2A5C
:100500002A2A2A2A2A2A2A2A2A2A0056616C696457
:100510002063686F69636573206172653A205B319F
:100520005D2D5B31365D20286368616E6E656C20E1
:10053000312D31362900536574206F7574707574D0
:1005400020666F7220706F727420005B585D2061AE
:10055000626F7274206368616E67657320616E6498
:10056000206578697420525820636F6E6669670051
:100570005B535D20736176652073657474696E6783
:100580007320746F205258005B525D20726576654F
:1005900072742052582073657474696E6773207486
:1005A0006F2064656661756C747300557365206EA9
:1005B000756D62657273205B312D445D20746F2010
:1005C0006564697420706F727473205B452D515D92
:1005D00020666F722073657474696E677300202DD6
:1005E00020726563656976657220636F6E66696700
:1005F000757261746F722C20727820737720000AF4
:100600000A6F70656E4C52536E67200053657420FC
:1006100073657269616C2062617564726174653AB8
:10062000200056616C69642063686F696365733A82
:100630002031202D20342B34202F2032202D203823
:10064000202F2033202D20382B34202F2034202D14
:10065000203132202F2035202D2031322B34202FF5
:100660002036202D20313600536574204368616E9A
:100670006E656C20636F6E6669673A20005365741F
:100680002044617461726174652028302D32293AEA
:10069000200053657420486F70206368616E6E653A
:1006A0006C7320286D61782032342C207365706162
:1006B000726174656420627920636F6D6D61732966
:1006C0002076616C69642076616C75657320312DCC
:1006D0003235353A2000536574206368616E6E656B
:1006E0006C2073706163696E6720287831306B48C5
:1006F0007A293A200053657420524620706F77653E
:10070000722028302D37293A200053657420524634
:10071000206D6167696320286865782920652E67E8
:100720002E20307844454144463030443A2000532E
:1007300065742062617365206672657175656E63AC
:10074000792028696E20487A293A20005B5A5D207A
:10075000656E746572207265636569766572206383
:100760006F6E66696775726174696F6E2075746902
:100770006C79005B465D20646973706C61792061FF
:10078000637475616C206672657175656E63696509
:10079000732075736564005B525D2063616C6375E3
:1007A0006C6174652072616E646F6D206B65792079
:1007B000616E6420686F70206C697374005B495DC2
:1007C000207265696E697469616C697A6520736508
:1007D0007474696E677320746F20736B65746368DB
:1007E0002064656661756C7473005B585D2072658A
:1007F00076657274206368616E67657320616E64EC
:100800002065786974206D656E75005B535D20739B
:100810006176652073657474696E677320746F20E8
:10082000454550524F4D20616E64206578697420B3
:100830006D656E7500557365206E756D62657273BA
:10084000205B302D395D20746F20656469742070E1
:100850006172616D657465727300202D2053797328
:1008600074656D20636F6E66696775726174696F18
:100870006E000A0A6F70656E4C52536E672000510D
:1008800029204F7574707574206265666F726520DB
:100890006C696E6B20283D465329203A2000502970
:1008A00020536C617665206D6F64652028657870D3
:1008B0006572696D656E74616C293A20004F29205C
:1008C00054696D65642042494E44206174207374FC
:1008D000617274757020203A20004E292050504DCE
:1008E000206F7574707574206C696D69746564200F
:1008F000202020203A200044495341424C454400E6
:100900004D292050504D205253534920746F20637D
:1009100068616E6E656C202020203A20004C2920F2
:1009200050504D206D696E696D756D2073796E63E1
:10093000202875732920203A200044495341424C15
:100940004544004B29204661696C736166652062ED
:100950006561636F6E20696E74762E2028312D32AA
:10096000353573293A20004A29204661696C736144
:10097000666520626561636F6E2064656C617920D5
:1009800028302D323535203D3E20313073202D204A
:100990003135306D696E293A200049292046616958
:1009A0006C7361666520626561636F6E206672714B
:1009B0002E203A200048292050574D2073746F7024
:1009C0002064656C6179202020202020203A2000BE
:1009D00047292050504D2073746F702064656C61FE
:1009E00079202020202020203A200046292046611E
:1009F000696C736166652064656C617920202020D4
:100A00002020203A200050574D206368616E6E65AB
:100A10006C200066756E6374696F6E3A2000292041
:100A2000706F72742000506F776572546F776572C3
:100A300000445446205548462033322D62697420C4
:100A400031306368004F70656E4C52536E67525878
:100A5000206D696E6920342F36636800466C7974A6
:100A6000726F6E2F4F72616E6765525820554846FF
:100A70002038636800525820747970653A20004429
:100A8000697361626C656400487A00203D3D200016
:100A900043616C63756C61746564207061636B6540
:100AA0007420696E74657276616C3A200042292068
:100AB0004D6963726F202868616C66292050504D23
:100AC000202020203A00412920496E766572746505
:100AD000642050504D20696E20202020203A0030A4
:100AE00029204D7574652062757A7A657220286DAB
:100AF0006F73746C79293A003929205365726961E2
:100B00006C2062617564726174653A00736D617224
:100B100074506F7274004672536B79005472616E38
:100B200073706172656E740044697361626C6564B0
:100B30000038292054656C656D657472793A2020FF
:100B40002020202020003729204368616E6E656CCC
:100B500020636F6E6669673A202000362920446161
:100B60007461726174652028302D32293A2020206A
:100B700000352920486F70206368616E6E656C7364
:100B80003A2020202020003429204368616E6E65C1
:100B90006C2073706163696E673A202000332920EE
:100BA000524620706F7765722028302D37293A2001
:100BB0002020003229205246206D616769633A2067
:100BC0002020202020202020003129204261736530
:100BD000206672657175656E63793A202020000089
:100BE00000000700020100000304060000000000EE
:100BF00000000001020408102040800102040810D7
:100C00002001020408102004040404040404040263
:100C10000202020202030303030303000000002395
:100C2000002600290000000000250028002B0000FD
:100C3000000000240027002A0000E22D11241FBE1E
:100C4000CFEFD8E0DEBFCDBF13E0A0E0B1E0E2ED32
:100C5000F1E602C005900D92A83CB107D9F716E065
:100C6000A8ECB3E001C01D92AC38B107E1F71CE07D
:100C7000CCE3DCE004C02297FE010E94EB2ECA33D5
:100C8000D107C9F70E941E2E0C94E7300C94000087
:100C900080917105813019F482E080937105809113
:100CA0007105833019F484E0809371050895A89547
:100CB0000895DC01ED91FC910190F081E02D099502
:100CC00008952091720530917305382748E0C901D5
:100CD000880F991F37FF06C09C0151E2252750E17C
:100CE000352701C09C01415091F730937305209343
:100CF0007205089588E38093740580E092ECA1E08A
:100D0000B0E08093750590937605A0937705B09336
:100D1000780587E08093810580E091EAACEBB3E34E
:100D20008093790590937A05A0937B05B0937C0519
:100D300085E0809382058DEE9EEFADEABEED809357
:100D40007D0590937E05A0937F05B0938005E3E831
:100D5000F5E080E090E0863028F4DC01AE54BC4F32
:100D60002C9101C020E0219301968831910599F7DB
:100D700082E080939B058AE080939C05089580E043
:100D80009EECADEEB4E38093B9059093BA05A093C1
:100D9000BB05B093BC0580E090E0A0E0B0E5809397
:100DA000BD059093BE05A093BF05B093C005E1ECCF
:100DB000F5E080E081938F5F8031E1F70895A0E056
:100DC000B0E0E5EEF6E00C94B42ED82F0E9419297D
:100DD0006115710581059105C9F30E94572F109285
:100DE0007D0510927E0510927F0510928005C4E06B
:100DF000812C912C54018A94C0907D05D0907E0561
:100E0000E0907F05F0908005FE2CED2CDC2CCC24AE
:100E10000E94522FA50194010E94932E6C0D7D1DFE
:100E20008E1D9F1D60937D0570937E0580937F05C9
:100E300090938005C15001F7DD2309F450C003E809
:100E400015E0E801A12CB12C62E3C62ED12CE12CD7
:100E5000F12C8881882309F442C0B39419F40E94CC
:100E60007A063DC00E94522FA70196010E94932E40
:100E7000E1E0E60FA3E8B5E08A2F801B8A1520F495
:100E80008D918E13F9CFE9CF2091820530E0A0E15A
:100E9000B7E20E942B2E9B01AC01AE2FB0E00E9466
:100EA0003A2E4090790550907A0560907B057090BD
:100EB0007C05640D751D861D971D4090B9055090E9
:100EC000BA056090BB057090BC05461657066806CB
:100ED000790618F2E993A39488E1A812BACFCDB7A6
:100EE000DEB7E0E10C94D02E8436910520F4BC01ED
:100EF00080E090E017C09C018E3B910528F42A55B4
:100F00003109AAE0B0E00CC0823D910528F4245BD1
:100F10003109A4E6B0E004C02D5C3109A8E5B2E0D7
:100F20000E942B2EA4E6B0E09B01AC010E943A2E59
:100F3000089590E08C599F4F0E947407089561E0D6
:100F40008AE00E94C62960E08AE00E94FF29089595
:100F5000892B11F061E001C060E08AE00E94FF2966
:100F6000089560E089E00E94C62961E088E00E945F
:100F7000C62961E087E00E94C62960E082E00E9405
:100F8000C62961E084E00E94C629089542E050E04D
:100F900068E476E080E00E9449280895E3E0F0E00C
:100FA00089E080935700E491E67081E0E63009F033
:100FB00080E00895CF93DF93C82F0E94CE07882347
:100FC00081F0DFB781E080937005F8940E945706A6
:100FD00088E180936000C0936000C1110E945706B1
:100FE000DFBFDF91CF9108958F929F92AF92BF9212
:100FF000CF92DF92EF92FF92CF93FC01C0A5EC2F2E
:10100000E770F0E0E658FC4FA081B0E0C7FF03C0F6
:1010100024E130E002C02FE030E0FC0197A183E141
:10102000989FF0011124E25CFE4F80809180A280A5
:10103000B380A20FB31F20E43FE14DE750E00E94D0
:10104000452EA50194010E94712E8C2F887149F4C0
:1010500069017A01E0EDCE0EE7E0DE1EE11CF11C35
:101060001BC0C7FF05C060E47AE88CE29EE004C0C4
:1010700060E07EEE8AEB9BE069017A01F8EBCF0E2F
:10108000FBE0DF1EE11CF11CA50194010E94712E02
:10109000C20ED31EE41EF51EC701B60169517C4F76
:1010A0008F4F9F4F28EE33E040E050E00E94712EBA
:1010B000A8EEB3E00E943A2ECF91FF90EF90DF9020
:1010C000CF90BF90AF909F908F9008958F3F9105E4
:1010D00051F048F0811522E0920738F081159340D5
:1010E00030F482E0089580E0089581E0089583E07F
:1010F0000895A0E0B0E0EFE7F8E00C94BD2EEB011E
:101100008A01B82FB695A0E028813981F8012083A3
:101110002A813B8121832C813D8122832E813F8145
:101120002383688179814A815B812C813D81EE81B5
:10113000FF819F2F9295990F990F907C272F2370F5
:10114000922B252F2370220F220F922B232F2370F7
:101150002295207F922BF80194830B5F1F4F2896D6
:10116000AF5FBA1788F680FF24C0888199810E94FA
:101170006608D82E8A819B810E946608E82E8C81A1
:101180009D810E946608F82E8E819F810E946608CC
:10119000F0E4DF9EA001112490E1E99E900111246A
:1011A000242B282BE4E0FE9EB0011124262BF8010D
:1011B0002083CDB7DEB7E7E00C94D92E803223E050
:1011C000920708F1883E23E0920740F48F51934044
:1011D000E4E096958795EA95E1F70895803D27E04C
:1011E000920718F48C5D93400895883928E092079F
:1011F00068F4885C974074E0969587957A95E1F756
:101200008D509C4F089580E090E008958FEF93E01B
:1012100008958C30910540F4A4E0880F991FAA9599
:10122000E1F7885D9C4F0895843F23E0920718F40E
:1012300084529C4F0895811524E0920740F486570C
:10124000934FF4E0880F991FFA95E1F7089580E92C
:1012500098E008959C013695279525753575821B74
:10126000930B9C0123733373969587959695879579
:1012700083739373820F931F9C0154E036952795D7
:101280005A95E1F7280F391F2F703F7041E051E068
:10129000249FC001259F900D349F900D1124892F0C
:1012A00008955F98882319F00000289A02C0000072
:1012B000289800005F9A000008955F9A000083B1AB
:1012C0005F980000869581700895CF93DF93D82FA3
:1012D0005C9A5F985C98C8E08D2F80780E945109D5
:1012E000DD0FC150C9F75F98DF91CF9108958F77D7
:1012F0000E9465090895CF93DF93D82FC8E08D2F02
:1013000080780E945109DD0FC150C9F75F98DF91C5
:10131000CF910895CF93DF935F98C8E080E0D82FF6
:10132000DD0F0E945D098D0FC150C9F7DF91CF918C
:1013300008950E9477090E948A095C9A0895A1E0A5
:10134000B0E0E5EAF9E00C94C22E806869830E945F
:1013500065096981862F0E947B095C9A2196E2E0EB
:101360000C94DE2ECF93C0917D05C827E82FF0E0C6
:10137000EC58FA4F678589E70E949F096C2F8DE32F
:101380000E949F096C2F82E40E949F09CF910895CB
:1013900086E20E9499090895CF93DF93EC016C8156
:1013A0008CE10E949F096D818DE10E949F096E81F1
:1013B0008EE10E949F096F8180E20E949F096885EB
:1013C00081E20E949F09698582E20E949F096A85E5
:1013D00083E20E949F096B8584E20E949F096C85CD
:1013E00085E20E949F096D858AE20E949F096E85B1
:1013F0008EE60E949F096F858FE60E949F0968898B
:1014000080E70E949F09698981E70E949F096A8994
:1014100082E70E949F09DF91CF910895CF92DF92DA
:10142000EF92FF92CF93DF936B017C01C11488E3AD
:10143000D8068CE9E8068CE1F80628F5C701B60164
:1014400020E836E948E950E00E94712EE9016897EA
:1014500060E879E687E69FEF0E944D2E6C0D7D1DBA
:101460008E1D9F1DF2E0660F771F881F991FFA954A
:10147000D1F721E732E040E050E00E94712EF22ED9
:10148000E32E80E421C0C701B60120E03DE241E344
:1014900051E00E94712EE901689760E073ED8EECD7
:1014A0009EEF0E944D2E6C0D7D1D8E1D9F1D660FA3
:1014B000771F881F991F21E732E040E050E00E942B
:1014C000712EF22EE32E80E66C2F6F71680F85E788
:1014D0000E949F096E2D86E70E949F096F2D87E766
:1014E0000E949F09DF91CF91FF90EF90DF90CF9006
:1014F0000895682F8DE60E949F0908958F929F920C
:10150000AF92BF92CF92DF92EF92FF92CF93DF9391
:10151000D82F83E00E94990980936F0584E00E9490
:10152000990980936E0560E086E00E949F0961E062
:1015300087E00E949F096FE789E00E949F0965E0AC
:101540008AE00E949F0962E18BE00E949F0965E1A9
:101550008CE00E949F096DEF8DE00E949F0960E082
:101560008EE00E949F09DD2319F08BE291E008C014
:1015700020919B0533E1239FC0011124825C9E4F83
:101580000E94CC096CE880E30E949F096FE082E32F
:101590000E949F0962E483E30E949F0980919C0559
:1015A00087FF02C064E101C06AE084E30E949F09F2
:1015B0006AE285E30E949F096DE286E30E949F092B
:1015C00064ED87E30E949F0960E088E30E949F0921
:1015D00060E089E30E949F09D11109C0C0907D0598
:1015E000D0907E05E0907F05F090800507C0C5E9AA
:1015F000CC2EC1ECDC2EED2CCEEDFC2ECAE38F2CD4
:101600009924AA24BB24682D8C2F0E949F09682D41
:1016100085E08C0F0E949F09FE2CED2CDC2CCC2445
:10162000CF5FCE3361F76FEF83E40E949F096FEFC6
:1016300084E40E949F096FEF85E40E949F096FEF89
:1016400086E40E949F09DD2311F066E002C06091EC
:1016500081058DE60E949F0960E089E70E949F094D
:10166000609182058AE70E949F0960E083E70E94FB
:101670009F0960E084E70E949F09D11109C0609131
:10168000790570917A0580917B0590917C0504C065
:1016900060E071EA8CEB93E30E940E0ADF91CF9138
:1016A000FF90EF90DF90CF90BF90AF909F908F9082
:1016B000089561E087E00E949F0964E28EE70E943E
:1016C0009F0963E088E00E949F0960E088E00E9433
:1016D0009F0965E087E00E949F0962E085E00E9423
:1016E0009F0983E00E94990980936F0584E00E941E
:1016F000990980936E05089583E00E94990980936B
:101700006F0584E00E94990980936E0561E087E08F
:101710000E949F096AE070E080E090E00E943C290E
:101720000E94590B00000895CF92DF92FF920F9311
:101730001F93CF93DF931F92CDB7DEB7082F162FDD
:101740008EE399830E949F09F02EC02E9981D92E95
:101750008C2D8F19811738F4F60161916F018FE795
:101760000E949F09F5CF64E085E00E949F0983E015
:101770000E94990980936F0584E00E9499098093E3
:101780006E050E94192960936A0570936B0580931A
:101790006C0590936D0569E087E00E949F0981E0E8
:1017A000809371050F90DF91CF911F910F91FF9062
:1017B000DF90CF9008950F931F930E94940B809118
:1017C0007105813099F40E94192900916A051091E0
:1017D0006B0520916C0530916D05601B710B820BC0
:1017E000930B603A76488140910548F380917105EA
:1017F000813031F46EE971E080EE95E00E94052BB6
:101800001F910F9108950F931F938091710582305E
:1018100021F41092710581E020C080917105813022
:10182000D9F40E94192900916A0510916B05209145
:101830006C0530916D05601B710B820B930B613A47
:1018400076488140910540F061E087E00E949F0961
:101850001092710582E001C080E01F910F91089500
:10186000CF93DF93EC014AE050E06D2F70E080EE03
:1018700095E00E94D32B6EE280EE95E00E94D72A7D
:10188000BE0184E0769567958A95E1F76F707727BA
:101890004AE050E080EE95E00E94D32B6EE280EEAD
:1018A00095E00E94D72ABE016F7077274AE050E08A
:1018B00080EE95E00E94D32BDF91CF910895D82F31
:1018C000C0E0CD1780F42D9A64E670E080E090E0EF
:1018D0000E943C292D9864E670E080E090E00E9430
:1018E0003C29CF5FEECF6CE271E080E090E00E9497
:1018F0003C29E6CF0F931F93CF93DF93EC01062F84
:1019000015E0115051F0CE010E94CE30081741F081
:10191000602FCE010E94D630F4CF82E00E945F0C8F
:10192000DF91CF911F910F910895A0E0B0E0EBE916
:10193000FCE00C94B42E482E562EC0E0D0E0612C72
:10194000712CE12CF12C00E010E041100CC06090F3
:10195000D20586E4689E3001112459E1E52EF12C70
:1019600008EB15E01EC091E049120FC06090D2054F
:10197000E6E46E9E30011124FBE16F0E711C49E21A
:10198000E42EF12C04E715E00CC082E0481209C0F7
:1019900028E1622E77247394EE24E394F12C01ED78
:1019A00015E043018C0E9D1E109273051092720576
:1019B0003401A62CA818B12CC30101966C01AE14F9
:1019C000BF04A8F4A00EB11E511006C0C3010E94AE
:1019D000CE30F501808305C0F5016081C3010E940E
:1019E0007A0CF50180810E9461063601E2CFC301C5
:1019F000511018C0C3010E94CE30B82EC6010E94FB
:101A0000CE302B2D30E0322F2227282B80917205EB
:101A1000909173058217930779F4C0E0D0E05524C4
:101A2000539493CF3601609173050E947A0C6091B4
:101A30007205C6010E947A0CC05EDE4FC13E92E084
:101A4000D90708F482CF852DCDB7DEB7E0E10C943D
:101A5000D02E61E082E00E94950C089560E082E063
:101A60000E94950C8091D105853020F01092D1050F
:101A70000E94290D8091D1058093D205089561E0DF
:101A800080E00E94950C61E081E00E94950C089531
:101A900060E080E00E94950C882351F060E081E0D6
:101AA0000E94950C882321F080917405883349F0B9
:101AB0000E94BF060E947A0681E00E94DF060E9413
:101AC0003F0D0895882319F06AEA71E002C06EEABA
:101AD00071E080EE95E00E94052B0895FF920F9330
:101AE0001F93CF93DF9369EC7BE080EE95E00E943B
:101AF000B12A4091790550917A0560917B057091EA
:101B00007C052AE030E080EE95E00E94DA2B63EB62
:101B10007BE080EE95E00E94B12A40917D055091D6
:101B20007E0560917F057091800520E130E080EEB8
:101B300095E00E94DA2B6DE97BE080EE95E00E9453
:101B4000B12A4AE050E06091810580EE95E00E9464
:101B5000022C67E87BE080EE95E00E94B12A4AE023
:101B600050E06091820580EE95E00E94022C61E7D2
:101B70007BE080EE95E00E94B12AC3E8D5E0F12C2D
:101B80008E0188818823A9F0FF2031F061EB71E09C
:101B900080EE95E00E94D42A21964AE050E0F801B8
:101BA000608180EE95E00E94CB2BF394F8E1FF1268
:101BB000E7CF80EE95E00E94DF2A6BE57BE080EEC8
:101BC00095E00E94B12A4AE050E060919B0580EECA
:101BD00095E00E94022C66E47BE080EE95E00E9496
:101BE000B12AE0919C05E770F0E0EE0FFF1FEE5781
:101BF000FC4F6081718180EE95E00E94052B61E3CE
:101C00007BE080EE95E00E94B12A80919C0588716E
:101C1000883069F028F4811113C068E27BE00CC0C1
:101C2000803141F0883161F46CE07BE005C06CE10B
:101C30007BE002C066E17BE080EE95E00E94F32A43
:101C400068EF7AE080EE95E00E94B12A4091750538
:101C50005091760560917705709178052AE030E023
:101C600080EE95E00E94DA2B6FED7AE080EE95E051
:101C70000E94B12A8091BD0580710E94620D66ECC0
:101C80007AE080EE95E00E94B12A8091BD058074D3
:101C90000E94620D6DEA7AE080EE95E00E94B12A22
:101CA0008091BD0580720E94620D60E97AE080EE4D
:101CB00095E00E94B12A84E795E00E94F407AB0109
:101CC000BC012AE030E080EE95E00E94BC2B6BE87E
:101CD0007AE080EE95E00E94B12A84E795E00E94C8
:101CE000F4079B01AC0160E472E48FE090E00E9495
:101CF000712EBA01A9012AE030E080EE95E00E9441
:101D0000BC2B68E87AE080EE95E00E94F32ACDB71C
:101D1000DEB7E5E00C94DB2E8F929F92AF92BF92DC
:101D2000CF92DF92EF92FF92811107C06FE77AE0C6
:101D300080EE95E00E94F32A2FC090E00E94740785
:101D400024E630E040E050E00E94712ECA01B90163
:101D50002AE030E040E050E00E94712E49015A0133
:101D60006B017C012AE030E0B501A40180EE95E032
:101D70000E94BC2B6EE280EE95E00E94D72A2AE0FA
:101D800030E0B701A60180EE95E00E94BC2B63E72E
:101D900080EE95E00E94172BFF90EF90DF90CF90A0
:101DA000BF90AF909F908F9008951F93CF93DF9334
:101DB00065E77AE080EE95E00E94B12A80919D056A
:101DC000813041F46CE57AE080EE95E00E94F32AE0
:101DD00010E050C0823019F465E47AE0F5CF843029
:101DE00019F461E37AE0F0CF853091F766E27AE0AA
:101DF000EBCFC12FD0E0C930D1050CF441C068E36E
:101E0000610F80EE95E00E94D72A6EE17AE080EEC5
:101E100095E00E94B12ABE016F5F7F4F4AE050E01B
:101E200080EE95E00E949B2B63E17AE080EE95E0E6
:101E30000E94B12AC356DA4FE981E03218F566E014
:101E40007AE080EE95E00E94B12A8981803130F0FD
:101E50006DE673E080EE95E00E94D42A69816F7090
:101E600070E06F5F7F4F4AE050E080EE95E00E94A7
:101E7000A42B1F5F80914605181708F4BACF0FC036
:101E800061E3BECFEF70F0E0EE0FFF1FEE56FC4FA8
:101E90006081718180EE95E00E94052BEACF6BEEA8
:101EA00079E080EE95E00E94B12A8091B5050E940C
:101EB0008C0E60ED79E080EE95E00E94B12A809171
:101EC000B6050E948C0E65EB79E080EE95E00E94ED
:101ED000B12A8091B7050E948C0E6AE979E080EE04
:101EE00095E00E94B12A4091AD055091AE056091F8
:101EF000AF057091B005411551056105710539F1C6
:101F00002AE030E080EE95E00E94DA2B67E679E087
:101F100080EE95E00E94B12A8091B1050E94990758
:101F2000AB01BC012AE030E080EE95E00E94DA2BA4
:101F300063E479E080EE95E00E94B12A4AE050E047
:101F40006091B20580EE95E00E94022C06C06AE323
:101F500079E080EE95E00E94F32A6DE179E080EE71
:101F600095E00E94B12A6091B3057091B4054AE0F2
:101F700050E080EE95E00E94EC2B60E079E080EE8E
:101F800095E00E94B12A6091AC05603450F470E095
:101F90006F5F7F4F4AE050E080EE95E00E94A42BF7
:101FA00006C067EF78E080EE95E00E94F32A6AEDC4
:101FB00078E080EE95E00E94B12A8091AB0580FF29
:101FC00003C063EB71E002C067EB71E080EE95E067
:101FD0000E94052B6DEB78E080EE95E00E94B12A1F
:101FE0008091AB0582700E94620D6EE978E080EE10
:101FF00095E00E94B12A8091AB0584700E94620D29
:102000006FE778E080EE95E00E94B12A8091AB0501
:1020100088700E94620DDF91CF911F9108950F93F8
:102020001F93CF93DF93209143052F3FA9F56FEFC7
:1020300075E080EE95E00E94B12A84E893E00E946A
:10204000300C6EED75E080EE95E00E94B12A809133
:102050004405909145050E94300C6BEA75E080EED6
:1020600095E00E94F32A68E875E080EE95E00E9412
:10207000F32A60E775E080EE95E00E94F32A6BE4B6
:1020800075E080EE95E00E94F32A80EE95E00E94D4
:10209000DF2A0E94D50E68C012160CF065C03327E7
:1020A00027FD30958091460590E0821793070CF448
:1020B0005BC066E375E080EE95E00E94B12A609116
:1020C0004305772767FD70954AE050E080EE95E084
:1020D0000E94A42B6BE075E080EE95E00E94B12A8F
:1020E00010E008E2809147051817D0F5C12FD0E025
:1020F000CC0FDD1FC85BDA4F288130E080914305AB
:10210000992787FD909501972817390739F56BEBCB
:1021100071E080EE95E00E94D42A4AE050E0602F02
:1021200080EE95E00E94CB2B6FEB71E080EE95E0A6
:102130000E94D42AE981EF70F0E0EE0FFF1FEE5607
:10214000FC4F6081718180EE95E00E94D42A63EC9F
:1021500071E080EE95E00E94D42A0F5F1F5FC2CF2E
:1021600080EE95E00E94DF2ADF91CF911F910F91C1
:102170000895FF920F931F93CF93DF93C3E8D5E0A9
:10218000F12C8E0188818823D1F165EC71E080EE1D
:1021900095E00E94D42A4AE050E06F2D80EE95E051
:1021A0000E94CB2B62ED71E080EE95E00E94D42A74
:1021B0002196F801208130E0A0E1B7E20E942B2EA9
:1021C0009B01AC01A0918205B0E00E943A2EAB01C8
:1021D000BC018091790590917A05A0917B05B09121
:1021E0007C05480F591F6A1F7B1F2AE030E080EEF4
:1021F00095E00E94DA2BF394F8E1FF12C2CFCDB73D
:10220000DEB7E5E00C94DB2E1092DD0485E6EEED02
:10221000F4E0DF011D928A95E9F70895CF93C82F66
:102220008F3719F0883009F045C0E091DD04EE23C6
:10223000D9F1E150E093DD04F0E0E252FB4F10826F
:102240006DE070E080EE95E00E945906C0E080915C
:10225000DD04C81760F4EC2FF0E0E252FB4F608120
:1022600070E080EE95E00E945906CF5FF0CF60E20B
:1022700070E080EE95E00E9459066DE070E080EE1F
:1022800095E00E945906C0E08091DD04C81778F5FA
:10229000EC2FF0E0E252FB4F608170E080EE95E0C1
:1022A0000E945906CF5FF0CF67E080EE95E00E9474
:1022B000D72A1DC08B3119F40E9404111AC08D3029
:1022C000C1F08A30B1F08091DD04843668F76C2F5C
:1022D00070E080EE95E00E945906E091DD0481E017
:1022E0008E0F8093DD04F0E0E252FB4FC08380E06C
:1022F00001C081E0CF910895CF93C82F0E94192982
:102300006093C6047093C7048093C8049093C90473
:10231000C093DB04CC2329F040E051EE60E070E094
:1023200004C040E855E260E070E080EE95E00E9475
:10233000612DCF9108959091CA04492F4F7050E0BC
:10234000BA016F5F7F4F292F30E0E4E03595279584
:10235000EA95E1F76217730759F0FA01E553FB4F6D
:10236000808381E0890F8F70907F892B8093CA04CE
:1023700008956EE770E080EE95E00E94590608959A
:10238000A3E1B1E0E6ECF1E10C94B52EE3E8F5E071
:10239000712C8191882321F0739428E17212F9CF76
:1023A00066ED71E080EE95E00E94052B4AE050E07A
:1023B000672D80EE95E00E94022C80E00E947E0A4C
:1023C0000E94590B8E010E5F1F4FC12CD12C76013C
:1023D000C39466246A945C2C0E940D294B015C0115
:1023E0002091820530E0A0E1B7E20E942B2E9B01F4
:1023F000AC01C701B6010E944D2E209179053091A4
:102400007A0540917B0550917C05620F731F841FF4
:10241000951F2091B9053091BA054091BB055091A7
:10242000BC05261737074807590718F4F8016082DA
:1024300025C08C2D0E94B20961E070E080E090E040
:102440000E943C29F80110820E940D29681979091F
:102450008A099B09643F71408105910540F40E94FF
:10246000C809F8019081981778F78083EDCF50FE66
:1024700003C02C982D9A02C02C9A2D982FEFC21AC7
:10248000D20AE20AF20A0F5F1F4F8FEFC816D1047B
:10249000E104F10409F09FCFCE019395FC01D82E01
:1024A0007FEF68EC2E2F281B271510F051E056C047
:1024B000DE01129651E02FEF41E03D91321710F00E
:1024C000322F01C0452F5F5F5F3F11F0232FF5CF03
:1024D0004193242F30E0A1E0B0E0AC0FBD1FA20F6C
:1024E000B31F5C93413079F0DE01A20FB31F5C9300
:1024F000423049F0AFEFBFEFAC0FBD1FA20FB31FCB
:102500006C934E3F78F6A2E0B0E0AC0FBD1FA20F77
:10251000B31F7C934D3F30F6A3E0B0E0AC0FBD1F7E
:10252000A20FB31F6C93BECF452F242F30E0FC01C8
:10253000E20FF31F6081AFEFB0E0AC0FBD1FA20F41
:10254000B31F2C91621748F44150DC01A40FB11D58
:102550002C9120836C934111E8CF5F5F571520F3D6
:10256000372D369520E0231770F4DC01A20FB11D42
:102570004C91522F530FFC01E50FF11D50815C93DC
:1025800040832E5FF0CFF3E8EF2EF5E0FF2E8C01B5
:10259000802F8D19871598F4F801C1908F014AE0BA
:1025A00050E06C2D80EE95E00E94CB2B6CE280EE2B
:1025B00095E00E94D72AF701C1927F01E9CF80EE12
:1025C00095E00E94DF2A81E0CD5EDE4FEFE00C94C3
:1025D000D12E1F920F920FB60F9211240F931F93BB
:1025E0002F933F934F935F936F937F938F939F931B
:1025F000AF93BF93EF93FF934091BD055091BE05FC
:102600006091BF057091C00589B18A019B0100747A
:1026100011272227332783FB882780F990E0A0E049
:10262000B0E0081719072A073B0709F468C0809132
:102630008400909185001092850010928400209172
:10264000A70421115CC045FD02C096958795853C85
:1026500029E09207C0F180910A0190E0A0E0B0E08B
:102660000CE176956795579547950A95D1F74115F1
:1026700051056105710521F441E050E060E070E032
:10268000481759076A077B07D8F480910A018F3FE2
:10269000B9F040E080910A01481780F4842F90E05F
:1026A000880F991FFC01E957FB4F20813181FC0104
:1026B000E55FFE4F318320834F5FECCF1092A8047B
:1026C00010920A011CC08D3B22E09207A8F02091D5
:1026D0000A01203188F410910A0121E0210F209392
:1026E0000A010E94DE08E12FF0E0EE0FFF1FE9571C
:1026F000FB4F9183808303C08FEF80930A01FF918A
:10270000EF91BF91AF919F918F917F916F915F9169
:102710004F913F912F911F910F910F900FBE0F90EE
:102720001F90189583E0809380008AE18093810058
:102730008FEF9FEF909389008093880010926F0035
:1027400088E080936D00E8E6F0E08081846080831B
:102750000895CF93DF930E942E0D8091D20584308F
:1027600039F585E00E94322AC1E0D0E0892B11F4CE
:10277000C0E0D0E086E00E94322A892B19F082E086
:1027800090E002C080E090E08C2B9D2B8230910580
:1027900039F08330910539F0019739F481E006C0B2
:1027A0001092D20505C082E001C083E08093D2057B
:1027B000DF91CF9108956F3018F086958058089575
:1027C00089E0689F802D11240895A0E0B0E0EBEE31
:1027D000F3E10C94BC2EC82F0E94192900913804F3
:1027E0001091390420913A0430913B046B017C0133
:1027F000C01AD10AE20AF30A9701860149E8C41611
:1028000043E1D406E104F10410F010923C0460931B
:1028100038047093390480933A0490933B042091D8
:10282000A7048FEF820F8230D8F5E0913C04EE23AD
:1028300009F44EC1E13011F482E0B8C1E03108F092
:1028400034C181E08E0F80933C04F0E0E957FB4FE8
:10285000C083803109F0ACC1E9E8F4E0213029F40B
:10286000A181A695A695808108C080819181A92F1C
:10287000A695A695A69596958795A03148F4B0E0C3
:1028800090E0AA0FBB1FA55FBE4F11969C938E933D
:102890001092A804329684E0E739F807F9F688C167
:1028A000233009F005C1E0913C04E11104C0CF30B0
:1028B00009F07EC10DC1E83148F481E08E0F8093AC
:1028C0003C04F0E0EA57FB4FC08372C1E83109F0E5
:1028D000ECC0C111EAC040E050E0ABE0CA01B3E097
:1028E000880F991FBA95E1F7A49F9001A59F300D1D
:1028F0001124F901E957FB4F6081E1817E2F777048
:1029000075956795FC01EE0FFF1FE55FFE4F718324
:102910006083F901E857FB4FB081B695B695B6953F
:10292000E181FE2FF295FF0FF07E6F2F6B2BE69566
:10293000E695E6957E2F777075956795FC01EE0F0D
:10294000FF1FE35FFE4F71836083F901E757FB4F81
:10295000B081B295B695B695B370C181DC2FDD0F0D
:10296000DD0F6D2F6B2BC295C695C695C370E281A6
:10297000E170EE0FEE0F7E2F7C2B75956795FC01B5
:10298000EE0FFF1FE15FFE4F71836083F901E55792
:10299000FB4FB081B695E181FE2FF795FF27F795A4
:1029A0006F2F6B2BE6957E2F777075956795FC01E1
:1029B000EE0FFF1FEF5EFE4F71836083F901E45756
:1029C000FB4FB081B295BF70E181FE2FF295F07F91
:1029D0006F2F6B2BE295EF707E2F77707595679553
:1029E000FC01EE0FFF1FED5EFE4F71836083F90166
:1029F000E357FB4FB081BB1FBB27BB1FC181DC2F3F
:102A0000DD0F6D2F6B2BCC1FCC27CC1FE281E37029
:102A1000EE0F7E2F7C2B75956795FC01EE0FFF1F47
:102A2000EB5EFE4F71836083F901E157FB4FB0818C
:102A3000B695B695E181FE2FF295FF0FFF0FF07C62
:102A40006F2F6B2BE695E6957E2F777075956795C2
:102A5000FC01EE0FFF1FE95EFE4F71836083F901F9
:102A6000E057FB4F20812295269527703181E32F77
:102A7000EE0FEE0FEE0F6E2F622B732F7295769581
:102A8000777075956795FC01EE0FFF1FE75EFE4FAF
:102A9000718360834F5F5F4F4230510509F01ECF55
:102AA00080919D0483FF1092A80410923C0480C082
:102AB000243009F07DC060913C0461110BC0C83A1C
:102AC000B1F4109273051092720588EA0E946106B3
:102AD00081E06CC0613019F4C093370404C06230E7
:102AE00031F4C09336048C2F0E9461065AC0E091E5
:102AF00036042E2F30E0220F331F462F50E0C9013D
:102B00000296841795073CF0633268F7FA01EC5798
:102B1000FB4FC083E8CF2D5F3F4F8C2F90E060913B
:102B20007205709173054217530749F4982F88274F
:102B300086279727909373058093720532C0681794
:102B4000790769F580913704813049F5E13118F052
:102B500080E180933604F0903604C8E8D4E000E0C9
:102B600010E00F15D0F4FE013197808190E0982F8E
:102B700088272881822B43E0969587954A95E1F72F
:102B80000E94DE08F801EE0FFF1FE55FFE4F918304
:102B900080830F5F1F4F2296E4CF1092A8041092FB
:102BA0003C0480913C04882319F08F5F80933C049F
:102BB000CDB7DEB7E8E00C94D82ECF93DF93E82FA3
:102BC000F0E0E854FA4FE185E03150F4F894F0E099
:102BD000EE0FFF1FE55FFE4F8081918178945DC00D
:102BE0008EE08E0F8B3058F4F0E0E25FF10924E6BE
:102BF0002E9FC0012F9F900D11240C964EC0E03FD8
:102C000009F446C038F4E13181F0E23191F0E0316D
:102C100039F409C0ED3FB1F1EE3FB9F1E13F79F18F
:102C200080E092E03AC082E101C083E10E945B2A29
:102C300034C085E00E94322AC1E0D0E0892B11F433
:102C4000C0E0D0E086E00E94322A892B19F082E0B1
:102C500090E002C080E090E08C2B9D2B82309105AB
:102C600041F08330910541F00197A9F086EA92E0A6
:102C700014C08CE090E011C089E591E00EC086E0C0
:102C800090E00BC08AEF93E008C08FEF93E005C09F
:102C900080E090E002C084EF93E0DF91CF9108954F
:102CA000A2E2B0E0E6E5F6E10C94B22E9E012F5FC1
:102CB0003F4F80E1D9011D928A95E9F764E072E007
:102CC00080EE95E029A33AA30E94052B0E947C0B7D
:102CD0001D8A1E8A1F8A188E312C212C00E0812C1F
:102CE000912C5401412C74E7572E7BE8672E72E338
:102CF000772EE0E5CE2EE3ECDE2EE12CF12C84EFF6
:102D000091E0A0E0B0E08D8F9E8FAF8FB8A380E000
:102D10009EECADEEB4E3898F9A8FAB8FBC8F80E0D1
:102D200094E7ABE8B2E3898B9A8BAB8BBC8B80EEDC
:102D300095E00E94192C892B09F4E1C080EE95E002
:102D40000E94462C9C0133272C32310509F442C0E5
:102D5000ACF42332310509F0ABC019821A821B8210
:102D60001C821D821E821F82188619861A861B8667
:102D70001C861D861E861F86188A60C02434310575
:102D800029F02335310509F4B2C092C064E480EE25
:102D900095E00E94D72A2AE030E040E054E76BE853
:102DA00072E380EE95E00E94652B6CE280EE95E088
:102DB0000E94D72A2AE030E040E05EEC6DEE74E33A
:102DC00080EE95E00E94652B6CE280EE95E00E941B
:102DD000172BADCF0F5F043009F0A9CF29813A81BD
:102DE0004B815C81A8EEB3E00E943A2E698B7A8B0E
:102DF0008B8B9C8B2D813E814F8158850E943A2E72
:102E0000698F7A8F8B8F9C8F29853A854B855C855E
:102E10002D8F3E8F4F8F58A32D853E854F85588926
:102E20000E943A2E6B017C0160323EE473078105FB
:102E3000910530F462E38CE10E949F0900E077CFB6
:102E4000603345E774078105910510F462E2F3CF22
:102E500060345CE975078105910510F466E2EBCFFB
:102E600080E5C81683ECD806E104F10410F462E1B1
:102E7000E2CF90E6C9169AEED906E104F10410F407
:102E800065E1D9CFA0E7CA16A1E1DA06A1E0EA061A
:102E9000F10410F461E0CFCFB0EACB16B6E8DB0660
:102EA000B1E0EB06F10410F463E0C5CF65E0C3CFF9
:102EB00010ED180F1A3008F03ACFE1E0F0E0EC0F17
:102EC000FD1F24E0029FE00DF11D112420813181BE
:102ED00042815381AAE0B0E00E943A2E610F711D39
:102EE000811D911D608371838283938320CF4988E4
:102EF0005A886B887C88812C912C540118CF8114BE
:102F00009104A104B10489F4C301B2010E940E0A24
:102F100061E070E080E090E00E943C291D8A1E8AFA
:102F20001F8A188E312C22242A948D8D9E8DAF8D70
:102F3000B8A188169906AA06BB06D0F40E94C80953
:102F40002D893E894F89588D280F311D411D511DF6
:102F50002D8B3E8B4F8B588F381608F4382E8215E8
:102F600008F4282E3FEF831A930AA30AB30A56C027
:102F7000C301B20128EE33E040E050E00E94712E20
:102F8000BA01A9012AE030E080EE95E00E94BC2B56
:102F90006CE280EE95E00E94D72A4AE050E0632D73
:102FA00080EE95E00E94CB2B6CE280EE95E00E94D3
:102FB000D72A6D897E898F89988DA50194010E94F9
:102FC000712EBA01A9012AE030E080EE95E00E945E
:102FD000BC2B6CE280EE95E00E94D72A4AE050E0DC
:102FE000622D80EE95E00E94CB2B6CE280EE95E0A6
:102FF0000E94172B4C0C5D1C6E1C7F1C898D9A8DBA
:10300000AB8DBC8D84159505A605B70520F44988C0
:103010005A886B887C88812C912C540129893A89A3
:103020004B895C89283E33404105510509F07FCE2C
:10303000A296E2E10C94CE2EACE1B0E0E2E2F8E13F
:103040000C94BC2E0E9419296B017C0181E00E9426
:103050007E0A14E703E0198361E0CE0101960E9425
:10306000DB0B009371050E94590B6AEF70E080E062
:1030700090E00E943C2980917105833089F480EEB4
:1030800095E00E94192C892B59F40E9419296C197A
:103090007D098E099F096038734C894C9140D8F2A4
:1030A00080917105833009F44FC08FE70E94770942
:1030B0000E948A098983843511F083E05CC00E94F4
:1030C0008A0910924405809345050E948A0920913F
:1030D000440530914505280F311D30934505209357
:1030E00044050E948A09809346050E948A098093BC
:1030F0004705813110F7F12C0F2D10E08091470525
:1031000090E0880F991F0817190740F40E948A0958
:10311000F801E85BFA4F8083F394EECF80E7898370
:1031200061E0CE0101960E94DB0B83E08093710584
:103130000E94590B62E370E080E090E00E943C291D
:1031400080917105833011F482E015C08FE70E94F1
:1031500077090E948A098983803509F0AECF0DE98D
:1031600015E00E948A09F80181938F01F5E0083B80
:103170001F07B9F781E06C96E8E00C94D82E809197
:103180004305992787FD9095A92FB92FFC0131960A
:10319000EB30F10508F066C0EC5CFF4F0C94E92EB3
:1031A00062E778E080EE95E00E94F32A84E893E0FD
:1031B0000E94300C6AE578E080EE95E00E94F32AE8
:1031C00065E378E080EE95E00E94F32A6BE078E01A
:1031D00080EE95E00E94F32A6AEE77E080EE95E0BB
:1031E0000E94F32A6DEB77E080EE95E00E94F32ACF
:1031F00067E977E080EE95E00E94F32A63E777E0E5
:1032000080EE95E00E94F32A6CE477E080EE95E092
:103210000E94F32A80EE95E00E94DF2A0E946E0D44
:1032200021C06FE277E01AC06AE077E017C065EF6F
:1032300076E014C066ED76E011C062E976E00EC07B
:103240006DE776E00BC068E676E080EE95E00E94E0
:10325000F32A62E276E002C06CE076E080EE95E070
:103260000E94F32A6AE070E080E090E00E943C292E
:1032700080EE95E00E94192C892B29F080EE95E0D4
:103280000E94462CF5CF0895ACE1B0E0EAE4F9E104
:103290000C94BC2E909143059F3F09F023C1482F09
:1032A00050E0FA013A97EF36F10508F00FC1E15C02
:1032B000FF4F0C94E92E61E172E0A0C06DE172E075
:1032C00080EE95E00E94052B85E789838BE1EDE98F
:1032D000F5E0DE01129601900D928A95E1F76CE11E
:1032E000CE0101960E94DB0B0E94590B83E0809374
:1032F000710568EC70E080E090E00E943C298091CC
:103300007105843009F0E2C08FE70E9477090E94BE
:103310008A098983853509F0D9C06DEE74E080EEA5
:1033200095E00E94F32A6FEC74E080EE95E00E9435
:10333000F32A61EB74E096C065E372E080EE95E0FD
:103340000E94052B89E6898361E0CE0101960E94E7
:10335000DB0B0E94590B83E08093710568EC70E0F1
:1033600080E090E00E943C2980917105843009F052
:10337000ADC08FE70E9477090E948A0989838E0178
:103380000E5F1F4F7E014DE1E40EF11C0E948A0981
:10339000F80181938F01EE15FF05C1F78BE1FE0166
:1033A0003296ADE9B5E001900D928A95E1F78981F9
:1033B000893409F08BC063E974E080EE95E00E94E7
:1033C000F32A65E774E080EE95E00E94F32A67E552
:1033D00074E048C06FE472E080EE95E00E94052B37
:1033E0008EEF8093430572C0805287508053909136
:1033F0004605981708F066C06EE572E080EE95E02D
:103400000E94052B63C084E18093430560E274E071
:1034100029C085E18093430569EE73E023C086E10E
:103420008093430562EB73E01DC087E18093430501
:1034300068E673E017C088E18093430567E573E0B1
:1034400011C089E18093430563E473E00BC08AE116
:10345000809343056EE273E005C08BE180934305E2
:1034600066E073E080EE95E00E94F32A2FC06CEED8
:1034700072E080EE95E00E94F32A8091AB0591E026
:103480001DC066ED72E080EE95E00E94F32A809107
:10349000AB0592E013C061EC72E080EE95E00E9413
:1034A000F32A8091AB0594E009C066EA72E080EEF1
:1034B00095E00E94F32A8091AB0598E089278093DC
:1034C000AB058FEF809343050E940F1080EE95E0CF
:1034D0000E94192C892B09F45AC180EE95E00E94B4
:1034E000462CF4CF0E940E11882309F450C180911C
:1034F000DD04811104C08FEF8093430540C140E09B
:1035000050E060E070E08EED94E00E94602F40910A
:103510004305042F112707FD1095212F312FF801A6
:103520003197EB31F10508F01AC1E255FF4F0C94C9
:10353000E92E552747FD50952091460530E0241788
:1035400035070CF40CC18B019C01015011092109B4
:103550003109003211052105310558F0C0904705A9
:10356000E9E4F5E0F12CD12CA8E2EA2E4150510912
:103570000FC0FA01E356FA4F61506083D8C0DF01F3
:1035800011972C9130E02417350729F0F3943296E7
:10359000FC10F5CFCAC00E2D10E020E030E0061779
:1035A00017072807390741F42081DA01A356BA4FDB
:1035B00011962C93DD24D394E394E8CF6F3F7105EB
:1035C0008105910511F008F0CAC06093B505AFC040
:1035D0006F3F71058105910511F008F0C0C060933F
:1035E000B605A5C06F3F71058105910511F008F082
:1035F000B6C06093B7059BC02091DE0420622037DF
:10360000E9F440E050E060E070E08FED94E00E946B
:10361000602F9B01AC01DC01CB010197A109B1092D
:103620000897A105B10508F0ADC0A4EDB0E30E9474
:103630003A2E6A5E7C4A8A46954E24C02636E9F4C4
:1036400040E050E060E070E08FED94E00E94602F79
:103650009B01AC01DC01CB010197A109B1090797DE
:10366000A105B10508F08EC0A8EAB1E60E943A2E85
:10367000645E7C438E46944E05C0611571058105DC
:10368000910571F08B019C0114572B483243013096
:10369000FAE51F07F2E62F07F2E03F0708F05FC0E8
:1036A0006093AD057093AE058093AF059093B00520
:1036B0003EC06F3F71058105910511F008F04FC0C4
:1036C0006093B10534C08B019C010150110921099F
:1036D00031090F3F11052105310508F040C0609305
:1036E000B20525C08B019C01045C194021093109F8
:1036F0000D344DE114072105310528F47093B4050C
:103700006093B30514C0611571058105910521F41D
:103710008FEF8093AC050BC0613471058105910575
:10372000F0F461506093AC0502C0DD20C1F08091DF
:10373000DC0481111AC080917D0590917E05A091D5
:103740007F05B09180050196A11DB11D80937D0577
:1037500090937E05A0937F05B093800506C060E737
:1037600072E080EE95E00E94052B0E9404118FEF1D
:10377000809343056AE080EE95E00E94172B0E943B
:103780000F1005C061E070E080E090E07BCF6C96A8
:10379000E8E00C94D82E6AE572E080EE95E00E9495
:1037A000F32A62E472E080EE95E00E94F32A80EE54
:1037B00095E00E94192C892B31F080EE95E00E9453
:1037C000462C0E9444190E941C18823029F0833034
:1037D00051F46DE072E002C064E272E080EE95E0C8
:1037E0000E94F32A08958FEF809343051092DC0422
:1037F0000E940F10809143058E3F69F080EE95E0A6
:103800000E94192C892BB1F380EE95E00E94462C82
:103810000E944419EFCF08950F931F931091430511
:103820001F3F09F0D2C0893409F457C000F588332E
:1038300009F469C058F4803309F477C008F061C016
:103840008B3109F440C08132B1F1B9C0813409F43F
:1038500087C030F4893309F466C0803461F1AFC0A9
:10386000823409F48EC0863409F448C0A8C0823678
:1038700009F487C078F4883531F128F48235C1F134
:103880008335E1F09CC08A3509F494C0813609F48F
:1038900067C095C0823761F128F4863679F18936A0
:1038A000E1F08DC0883779F08A3709F483C0833717
:1038B00009F085C003C061E172E015C00E943F0DB0
:1038C0006EE872E004C00E94480D68EA72E080EE83
:1038D00095E00E94052B8EEF70C00E947A060E9430
:1038E000BF0667EC72E080EE95E00E94052B67C092
:1038F00081E00E94DF0660EE72E0F5CF0E94B91011
:103900005EC080535AC06AEF71E080EE95E00E947D
:10391000F32A90919C0588E0890F8871977E892B06
:1039200080939C051AC089E048C067EE71E080EE84
:1039300095E00E94F32A8091BD059091BE05A0916B
:10394000BF05B091C00520E182278093BD0590930B
:10395000BE05A093BF05B093C005109343052FC0CB
:1039600061ED71E080EE95E00E94F32A8091BD0543
:103970009091BE05A091BF05B091C00540E4842799
:1039800010C060EC71E080EE95E00E94F32A809117
:10399000BD059091BE05A091BF05B091C00520E284
:1039A00082278093BD059093BE05A093BF05B09379
:1039B000C00502C00E94CB1B8FEF8093430580910E
:1039C00043058E3F09F0D4C0DDC00E940E1188234C
:1039D00009F4D8C08091DD04811104C08FEF809379
:1039E0004305C6C040E050E060E070E08EED94E03A
:1039F0000E94602F00914305112707FD1095212F8C
:103A0000312FF8013197E930F10508F0B4C0E753E0
:103A1000FF4F0C94E92E8B019C01015014472B4859
:103A200032430F3F19452246324008F0A4C060934C
:103A3000790570937A0580937B0590937C0577C018
:103A400060937D0570937E0580937F05909380053C
:103A500081E08093DC046BC06830710581059105BD
:103A600008F089C06093810562C08B019C01015000
:103A70001109210931090A3011052105310508F024
:103A80007AC06093820553C061EB71E08EED94E0E3
:103A90000E949A3010E0009799F00E9474300097CD
:103AA00079F0183130F4E12FF0E0EC58FA4F8787C5
:103AB0001F5F61EB71E080E090E00E949A30EBCFF5
:103AC0001831A8F5E12FF0E0EC58FA4F17861F5F88
:103AD000F7CF653071058105910508F04CC0609302
:103AE0009B0525C08B019C01015011092109310959
:103AF0000630110521053105F0F520919C05287F40
:103B0000262B20939C0513C08B019C0101501109A9
:103B1000210931090115124C2140310560F56093EE
:103B2000750570937605809377059093780580915D
:103B3000DC04811113C080917D0590917E05A091D8
:103B40007F05B09180050196A11DB11D80937D0573
:103B500090937E05A0937F05B09380050E94041189
:103B60008FEF809343056AE080EE95E00E94172B6B
:103B70000E94BF1807C060E772E080EE95E00E94E7
:103B8000052BECCF1F910F9108958FEF8093430584
:103B90001092DC040E94BF18809143058E3F69F0AB
:103BA00080EE95E00E94192C892BB1F380EE95E010
:103BB0000E94462C0E940C1CEFCF6AE070E080E06F
:103BC00090E00E943C2980EE95E00E94192C892B00
:103BD00029F080EE95E00E94462CF5CF0895CF9312
:103BE000C82F682F80EE95E00E94732C9091680595
:103BF0009C2790936805CF910895A1E0B0E0E3E0A1
:103C0000FEE10C94C22E99830E94EF1D9981892FA9
:103C10000E94EF1D2196E2E00C94DE2E1F93CF93BD
:103C2000DF93182FEB011092680565EB70E080EED2
:103C300095E00E94590662E670E080EE95E00E94F1
:103C40005906812F0E94EF1DCE010E94FD1DDF91BC
:103C5000CF911F9108956091680580EE95E00E94D4
:103C6000732C0895A1E2B0E0E8E3FEE10C94BE2ECF
:103C70007B018A018C3009F453C108F040C08630C2
:103C800009F4BCC018F5833009F491C070F4813098
:103C900009F472C0823009F048C26BE170E082E042
:103CA0000E940E1E0DE915E078C0843009F487C02B
:103CB000853009F03AC26091470570E0660F771FC2
:103CC00085E00E940E1E08E415E086C0893009F4E4
:103CD000A7C070F4873009F49BC0883009F025C272
:103CE00061E070E088E00E940E1E8091D20523C240
:103CF0008A3009F4CAC08B3009F4F2C016C28A3681
:103D000009F475C1D8F4873609F43AC138F4853618
:103D100009F40EC1863609F41FC107C2883609F4BA
:103D200037C1893609F001C261E070E089E60E947E
:103D30000E1E0E947A060E94BF06F5C18D3609F458
:103D4000D4C138F48B3609F491C18C3609F49AC188
:103D5000ECC18E3609F4DCC1873C09F0E6C161E0B4
:103D600070E087EC0E940E1E81E00E94EF1D0E9411
:103D70002B1E10926905E3C169E270E081E00E94A8
:103D80000E1E04E715E0F80181918F010E94EF1DDE
:103D9000F5E00D391F07B9F7D0C1F80181918F0106
:103DA0000E94EF1DF5E0083B1F07B9F7C6C161E0AF
:103DB00070E083E00E940E1E0E941C18BCC161E0EE
:103DC00070E084E00E940E1E81E00E94EF1D0E94C0
:103DD0002B1E0E945016B3C18091470590E0880FBA
:103DE000991F9801285435402817390708F0A5C1B4
:103DF000F80181918F010E94EF1DEECF62E070E02B
:103E000086E00E940E1E84E893E00E94FD1D95C18D
:103E100061E070E087E00E940E1E809146058BC134
:103E200086E6898361E0CE0101960E94DB0B0E9449
:103E3000590B83E08093710568EC70E080E090E0BE
:103E40000E943C29809171058430D9F48FE70E944B
:103E500077090E948A098983863469F460E270E0F8
:103E600089E00E940E1E10E20E948A090E94EF1D46
:103E70001150D1F762C161E070E089E00E940E1E2E
:103E800052C161E070E089E053C169E170E08AE00D
:103E90000E940E1E81E08093B805209170058091EC
:103EA000BD059091BE05A091BF05B091C00522232C
:103EB00011F0806801C08F778093BD059093BE0597
:103EC000A093BF05B093C00508EB15E0F801819100
:103ED0008F010E94EF1DF5E0013D1F07B9F72DC1CD
:103EE00061E270E08BE00E940E1E8091A8048F3F7B
:103EF00039F08091A80491E0980F9093A80402C033
:103F00008091A8040E94EF1D10E0812F0E94DD1512
:103F10000E9409090E94FD1D1F5F1031B1F70DC1FC
:103F200061E070E08CE00E940E1E8091D10503C11B
:103F300061E070E085E60E940E1E89E2E816F10459
:103F400009F0F8C0D801E4E7F5E08D91819385E0B0
:103F5000ED39F807D1F7E7C061E070E086E60E942E
:103F60000E1EEBE1EE16F10409F0E4C0D801EDE914
:103F7000F5E08D91819385E0E83BF807D1F7D3C058
:103F800061E070E087E60E940E1E0E943F0DCBC0EC
:103F900061E070E088E60E940E1E85E789838BE170
:103FA000EDE9F5E0DE01129601900D928A95E1F7B8
:103FB0006CE1CE0101960E94DB0B0E94590B83E05D
:103FC0008093710560E273E080E090E00E943C29FC
:103FD00080917105843009F0ADC08FE70E947709A8
:103FE0000E948A098983853509F0A4C09CC061E0DC
:103FF00070E08AE60E940E1E89E6898361E0CE01A8
:1040000001960E94DB0B0E94590B83E0809371059F
:1040100060E273E080E090E00E943C2980917105AD
:10402000843009F087C08FE70E9477090E948A09CF
:1040300089838E010E5F1F4F7E01EDE1EE0EF11CB4
:104040000E948A09F80181938F01EE15FF05C1F7DF
:104050008BE1FE013296ADE9B5E001900D928A95B3
:10406000E1F78981893409F065C05DC061E070E0E5
:104070008BE60E940E1EF80180818093D2050E947B
:10408000480D51C061E070E08CE60E940E1EF0E227
:10409000EF16F10461F487E6898380E2F801DE011E
:1040A000129601900D928A95E1F761E203C087E4D0
:1040B000898361E0CE0101960E94DB0B0E94590BBF
:1040C00083E0809371056CE474E080E090E00E94EE
:1040D0003C2980917105843069F58FE70E9477094A
:1040E0000E948A09873431F51EC061E070E08DE6D8
:1040F0000E940E1E89E1E816F104E1F4D801E8EB14
:10410000F5E08D91819385E0E13DF807D1F70BC093
:1041100061E070E08EE60E940E1EF80180818093BF
:10412000D1050E94290D81E006C061E070E08AECB3
:104130000E940E1E80E00E94EF1D0E942B1EA19681
:10414000E6E00C94DA2EA0E0B0E0E9EAF0E20C94AC
:10415000BC2ECAECD3E014E606E035E0F32E44E0D2
:10416000E42E53E0D52E62E0C62E80EE95E00E944C
:10417000192C892B09F49BC080EE95E00E94462CF7
:10418000282F809335044091340450E04730510586
:1041900060F7FA01EE52FF4F0C94E92E853B29F7A8
:1041A00081E080933404E1CF823609F07DC0C09273
:1041B0003404DBCF8093330480933204D0923404F0
:1041C000D4CF9C0133273093310420933004909155
:1041D0003204982790933204E0923404C6CF382FEB
:1041E00022274091300450913104242B352B3093F9
:1041F0003104209330049091320498279093320434
:10420000F09234042536310508F4AFCF61E070E058
:104210008CEC0E940E1E81E00E94EF1D0E942B1E5E
:1042200043C020912E0430912F04F901E653FC4F36
:10423000808390913204982790933204C9010196AB
:1042400090932F0480932E042091300430913104F8
:104250008217930708F489CF0093340486CF8091A6
:10426000320482130BC060912E0470912F044AEC2B
:1042700053E0809133040E94321E0DC062E070E072
:104280008BEC0E940E1E809133040E94EF1D8091E2
:1042900068050E94EF1DFE01812F11928A95E9F7B2
:1042A00010922F0410922E04109234045ECFCDB7DA
:1042B000DEB7E8E00C94D82E81E080936905809108
:1042C0006905882349F080EE95E00E94192C892B1E
:1042D000B1F30E94A320F3CF0895AAE2B0E0E3E790
:1042E000F1E20C94BA2E0E940D296B017C0181E051
:1042F0000E947E0A80EE95E00E94192C892B29F0FD
:1043000080EE95E00E94462CF5CF2D9811E072E6E4
:10431000B72EE9E2AE2E03E00E940D296C197D094B
:104320008E099F09693C710581059105D0F1112322
:10433000C1F10E940D296B017C012C9A80ED97E060
:104340000E94A807B982E4E7F5E0DE0112968A2D03
:1043500001900D928A95E1F76AE2CE0101960E94E2
:10436000DB0B2C9880E090E00E94A8070093710579
:104370000E94590B62E370E080E090E00E943C29CB
:1043800080917105843061F4009371058FE70E947C
:1043900077090E948A0911E0823419F410E001C003
:1043A00011E08BE00E94322A892B81F411E00EC0CB
:1043B0002D9A2C9A80EE95E00E94462C8D30910526
:1043C000A9F05CF40A9791F02D982C9880EE95E076
:1043D0000E94192C892B61F79FCF8332910579F0C8
:1043E0008234910589F70E945C21EECF62EB71E087
:1043F00080EE95E00E94F32A0E94C51DE5CF0E9441
:104400005016E2CF8F929F92AF92BF92CF92DF92DF
:10441000EF92FF921F93CF93DF938BE00E94322A9B
:10442000892B09F089C068EC70E080E090E00E9480
:104430003C2980E090E00E94A8070E940D294B01D2
:104440005C016B017C0180ECC80E82E1D81EE11C8E
:10445000F11C0E940D296C157D058E059F0530F419
:104460008BE00E94322A892BA1F364C08BE00E946A
:10447000322A892B09F05EC080ED97E00E94A807E0
:104480000E940D296B017C01D0E0C1E088E4880E18
:1044900086E2981EA11CB11C11E08BE00E94322A1A
:1044A000892B21F58C149D04AE04BF0430F480EDFB
:1044B00097E00E94A807D1E0F0CF0E940D296C1967
:1044C0007D098E099F09693C71058105910528F3D5
:1044D0000E940D296B017C01C12719F080ED97E046
:1044E00002C080E090E00E94A807D7CF80E090E073
:1044F0000E94A807DD23B9F08091D10590E00196D4
:1045000065E070E00E945D2E8093D1050E94290D28
:104510000E94A9130E94480D64EF71E080E090E0D2
:104520000E943C2909C080E00E94DF060E94C01161
:104530000E943F0D0E946D21DF91CF911F91FF904E
:10454000EF90DF90CF90BF90AF909F908F900895A5
:10455000CF92DF92EF92FF9280E00E94DA070E94F2
:10456000B10761E08DE00E94C62961E08CE00E9405
:10457000C62960E08BE00E94C62960E085E00E94C9
:10458000C62961E085E00E94FF2960E086E00E9484
:10459000C62961E086E00E94FF2960E083E00E9476
:1045A000C62961E083E00E94FF2961E08EE00E945D
:1045B000C62960E08EE00E94FF290E949F0740E02C
:1045C00052EC61E070E080EE95E00E94612D0E9467
:1045D000A9130E94480D0E9492138FEF8093A804A4
:1045E0000E94C60778940E940D296B017C0180917E
:1045F000A8048F3F59F40E940D296C197D098E097A
:104600009F09603D77408105910588F380ED97E033
:104610000E94A80761E08BE00E94FF292D9A80EE9E
:1046200095E00E94192C892B29F080EE95E00E94DC
:10463000462CF5CF6DEF72E080EE95E00E94D42A13
:1046400084E893E00E94300C64E173E080EE95E032
:104650000E94D42A4AE050E062E070E080EE95E0EB
:104660000E94A42B62E370E080E090E00E943C296D
:1046700080EE95E00E94192C04970CF180EE95E0F5
:104680000E94462C82349105D1F480EE95E00E9480
:10469000462C8E34910599F480EE95E00E94462CCC
:1046A0008434910561F480EE95E00E94462C819758
:1046B00031F480E090E00E94A8070E946D214091B3
:1046C0007505509176056091770570917805DB014D
:1046D000CA010197A109B1090497A105B10568F4C0
:1046E0004093A704433029F440EA56E861E070E0C3
:1046F00004C040E052EC61E070E080EE95E00E9482
:10470000612D0E9402222D9880E090E00E94A8076F
:104710000E9492131092C3048091BD0583FF11C0C3
:1047200080918905882351F080919005882331F08C
:1047300080919705882311F087E001C085E0809380
:10474000C30480E00E947E0A8091C4040E94B209E2
:104750000E94590B10923F0410923E0410923D04A7
:10476000F12C8091D2058F15B0F062E370E080E00B
:1047700090E00E943C2980ED97E00E94A80762E348
:1047800070E080E090E00E943C2980E090E00E9490
:10479000A807F394E6CF80919C0584FF08C0982F6A
:1047A000987181E0983109F080E00E947C118FE0DF
:1047B0000E94DA07FF90EF90DF90CF900895EF927C
:1047C000FF920F931F93CF93DF938C016EE770E0FE
:1047D00080EE95E00E945906E801F12CF0E2EF2E00
:1047E0008E0188818D57823048F46DE770E080EE4D
:1047F00095E00E94590688818E2588832196F801CC
:10480000608180EE95E00E94732CF394F9E0FF1232
:10481000E7CF6EE770E080EE95E00E945906CDB7D5
:10482000DEB7E6E00C94DA2EA9E0B0E0EAE1F4E2CB
:104830000C94C22E9091C50491110EC09EEF9983E5
:104840008A836B8350E0559547954C832D83198659
:1048500018861F821E822EC04091CA04842F90E0C9
:10486000B4E095958795BA95E1F7242F2F7030E045
:104870008217930719F18DEF89831B82FE0134960D
:1048800050E0842F90E0A4E095958795AA95E1F7F4
:10489000242F2F7030E08217930749F0DC01A553D5
:1048A000BB4F8C918193405F5F5F563051F74093CF
:1048B000CA045A83CE0101960E94DF238091C50469
:1048C00090E0019666E070E00E945D2E8093C50442
:1048D0002996E2E00C94DE2EA0E0B0E0E2E7F4E2FC
:1048E0000C94BB2E6C016EE770E080EE95E00E94A8
:1048F00059068601E12CF12CC0E0D0E030E2B32E65
:10490000F801608183E8860F823078F46DE770E00B
:1049100080EE95E00E945906F80160816B2570E0F9
:1049200080EE95E00E94590604C080EE95E00E945A
:10493000732CE114F10459F0F80180819E01280FD5
:10494000311DC901C92FDD27C80FD91FDD273FEF52
:10495000E31AF30A89E0E816F10459F028E0E216B8
:10496000F10421F48C2F8095F60180870F5F1F4F93
:10497000C7CFCDB7DEB7E9E00C94D72EA9E0B0E001
:10498000E4ECF4E20C94C22EE82F362F8091C5049B
:1049900090E0019664E270E00E945D2E8093C50471
:1049A00058E9598350E15A83813089F048F08230C8
:1049B000B9F08330D9F48B8381EF8C833D8319C0A8
:1049C00085E08B8381EF8C832F5F2D8312C08B83D7
:1049D00081EF8C8384E6489FA00111245D8309C088
:1049E00084E08B8381EF8C83ED8303C00E94B91137
:1049F00004C0CE0101960E946C242996E2E00C943A
:104A0000DE2EA2E0B0E0E7E0F5E20C94B72E182F1E
:104A1000762E2A8349830E9419296B017C0180919B
:104A2000DB048090C6049090C704A090C804B090A6
:104A3000C9042A8149818823C1F0D701C601881998
:104A40009909AA09BB094C015D0191EE89169EE204
:104A50009906A104B10420F1241708F4422F202F55
:104A6000672D812F0E94BE2413C0D701C60188196B
:104A70009909AA09BB094C015D0191E3891695E7E3
:104A80009906A104B10460F0672D812F0E941424BF
:104A9000C092C604D092C704E092C804F092C90440
:104AA0002296EDE00C94D32EA2E2B0E0EAE5F5E226
:104AB0000C94B82E8CE00E94990981110DC06CE114
:104AC00073E080EE95E00E94052B2D9A80E00E9415
:104AD0007E0A0E94590B2D9880EE95E00E94192CB9
:104AE000892B01F180EE95E00E94462C9091A7045D
:104AF000992319F00E94E513EFCF40913E0450E056
:104B00009A012F5F3F4F2F71332760913F0470E070
:104B10002617370709F3FA01E75BFB4F80832093E1
:104B20003E04DACF80917105843009F086C00E947E
:104B30001929611571058105910549F06093B50446
:104B40007093B6048093B7049093B8040CC081E0CE
:104B500090E0A0E0B0E08093B5049093B604A093F9
:104B6000B704B093B8048091AB049091AC04816019
:104B70009093AC048093AB0483E0809371058FE73E
:104B80000E94770909E614E00E948A09F8018193DE
:104B90008F01F4E002371F07B9F72091720480916A
:104BA0006904982F922796FF3BC090E49227909338
:104BB0007204982F98739833F1F410E0212F30E0AD
:104BC00080916904877090E0821793074CF11F5F12
:104BD00020919C05812F90E0FC01E759FB4F24FFB9
:104BE00004C080810E949B11E9CF608180EE95E036
:104BF0000E94732CE3CF8F7399F480916A048093A1
:104C0000B40480916B048093B20480916C0480930F
:104C1000B10480916F0490E09093AA048093A9045A
:104C200080913D04813019F482E080933D048091AD
:104C30003D04833011F410923D040E9419296B0148
:104C40007C018091AD049091AE04A091AF04B0912D
:104C5000B0040097A105B105C9F0A7019601281B72
:104C6000390B4A0B5B0BDA01C901883B9B40A1055C
:104C7000B10560F00E94C8098093B3041092AD049E
:104C80001092AE041092AF041092B0048091B90457
:104C90009091BA04A091BB04B091BC0446015701A5
:104CA000881A990AAA0ABB0A84E795E00E94F407C9
:104CB00086169706A806B90608F4B1C0C092B904D2
:104CC000D092BA04E092BB04F092BC040E94570652
:104CD0008091A8048830A0F08091BD059091BE0518
:104CE000A091BF05B091C0055CE1B695A7959795D9
:104CF00087955A95D1F7892B8A2B8B2B09F0B8C150
:104D00008091A8048F5F8093A8048091B50490914E
:104D1000B604A091B704B091B8040097A105B105FD
:104D2000F1F0C81AD90AEA0AFB0A84E795E00E9462
:104D3000F4076C157D058E059F0508F00FC1809165
:104D4000BD0584FD04C080ED97E00E94A807109285
:104D5000B5041092B6041092B7041092B804909162
:104D60007204907C9093720450913E0480913F04B1
:104D700020913D04581709F40EC1223009F00BC1EF
:104D8000905890937204E0919C05E770F0E0E6582B
:104D9000FC4F6081693008F0E6C0615040E0461386
:104DA000E4C080933F0487E3840F90917204892BC1
:104DB000809372044093400483E080933D042C9AD6
:104DC000109181058091C304811132C18091BD058C
:104DD00082FD3AC1812F0E94790A8091C4040E9409
:104DE000B209E0919C05E770F0E0E658FC4F608165
:104DF00082E794E00E94940B8091BD0582FD2DC155
:104E0000E091C404EF5FE093C404E83109F42DC1DC
:104E1000F0E0EC58FA4F8785882309F426C10E94F8
:104E2000030C813069F580919C05887149F180916E
:104E3000AB049091AC04880F991F9093AC048093BD
:104E4000AB0483E0809371050E94590B0E941929DD
:104E50006093AD047093AE048093AF049093B0045C
:104E6000672B682B692B61F481E090E0A0E0B0E053
:104E70008093AD049093AE04A093AF04B093B004BC
:104E800080919C0584FF1FC08091AB049091AC047D
:104E90008E7F0E942A09182F6091A9048091B40482
:104EA0000E94DB13482F612F8091B30449A30E9415
:104EB000DB130091D205282F49A16091B1048091A4
:104EC000B2040E9401252C988091C1048130C1F068
:104ED00018F08230B1F1D9C08BE00E94322A892BC0
:104EE00009F0D3C081E08093C1040E940D29609332
:104EF000BD047093BE048093BF049093C004C5C0EA
:104F00008BE00E94322A892B31F50E940D29C09036
:104F1000BD04D090BE04E090BF04F090C0046C19B2
:104F20007D098E099F09693E73408105910508F44A
:104F3000ACC082E08093C10480ED97E00E94A80796
:104F4000A4C08BE00E94322A892B09F49EC080E025
:104F500090E00E94A8071092C10497C080E090E002
:104F60000E94A807FCCE68E019CF851709F419CF75
:104F70004F5F242F30E090E0F901EE58FB4FDC0149
:104F8000A75BBB4F7C917083F901E05CFB4F7083A2
:104F900001968F7104CF2430B1F42091400481E454
:104FA00094E0A3E7B4E0FC013E2F381B321718F45D
:104FB00031913D93F9CF87E3820F90917204892B51
:104FC00080937204F9CE8091C104823051F49160D3
:104FD000909372042D9A8E010F5F1F4FF12CB80130
:104FE00010C02D9880913D04811103C081E0809311
:104FF0003D0480913D04833071F784E080933D044B
:10500000EACF8F2D69A37AA30E94DD15F801819361
:1050100091938F01F39469A17AA1F0E1FF12F1CF8E
:1050200080919C0543E754E087700E947908C7CEC1
:10503000112309F4CBCE9091C20421E0290F2093D3
:10504000C2049813C3CE1DC085E00E94322A892B6A
:1050500009F0C0CE2D9A17E0BDCE85E00E94322A1D
:10506000892B09F0CDCE2D98CBCE1092C404D7CE8B
:105070008091A804883009F42D9A89E08093A804CF
:10508000CECE1092C2041150A1CEA296ECE00C94A8
:10509000D42E8230E8F4E82FF0E0EE0FFF1FED523F
:1050A000FA4F71836083813041F0809169008C7F79
:1050B000842B80936900E89A089580916900440FD9
:1050C000551F440F551F837F842B80936900E99AF5
:1050D00008951F920F920FB60F9211242F933F93B2
:1050E0004F935F936F937F938F939F93AF93BF93F0
:1050F000EF93FF938091D3059091D405892B29F0EC
:10510000E091D305F091D4050995FF91EF91BF91FE
:10511000AF919F918F917F916F915F914F913F914F
:105120002F910F900FBE0F901F9018951F920F9206
:105130000FB60F9211242F933F934F935F936F936A
:105140007F938F939F93AF93BF93EF93FF93809140
:10515000D5059091D605892B29F0E091D505F091E0
:10516000D6050995FF91EF91BF91AF919F918F91D6
:105170007F916F915F914F913F912F910F900FBE53
:105180000F901F9018951F920F920FB60F92112437
:105190002F933F938F939F93AF93BF938091D805A5
:1051A0009091D905A091DA05B091DB053091D70532
:1051B00023E0230F2D3720F40196A11DB11D05C05A
:1051C00026E8230F0296A11DB11D2093D7058093D9
:1051D000D8059093D905A093DA05B093DB058091AB
:1051E000DC059091DD05A091DE05B091DF0501960B
:1051F000A11DB11D8093DC059093DD05A093DE0514
:10520000B093DF05BF91AF919F918F913F912F9107
:105210000F900FBE0F901F9018952FB7F8946091C4
:10522000D8057091D9058091DA059091DB052FBFE3
:1052300008953FB7F8948091DC059091DD05A09129
:10524000DE05B091DF0526B5A89B05C02F3F19F0FC
:105250000196A11DB11D3FBF6627782F892F9A2F78
:10526000620F711D811D911D42E0660F771F881F1F
:10527000991F4A95D1F70895CF92DF92EF92FF924E
:10528000CF93DF936B017C010E941929EB01C114BC
:10529000D104E104F10479F00E9419296C1B7D0B03
:1052A000683E7340A0F381E0C81AD108E108F10814
:1052B000C851DC4FECCFDF91CF91FF90EF90DF90A2
:1052C000CF900895789484B5826084BD84B5816060
:1052D00084BD85B5826085BD85B5816085BDEEE6FE
:1052E000F0E0808181608083E1E8F0E010828081DD
:1052F00082608083808181608083E0E8F0E080814B
:1053000081608083E1EBF0E0808184608083E0EB6A
:10531000F0E0808181608083EAE7F0E08081846052
:1053200080838081826080838081816080838081AE
:10533000806880831092C1000895833081F028F442
:10534000813099F08230A1F008958630A9F087303D
:10535000B9F08430D1F4809180008F7D03C08091BA
:1053600080008F7780938000089584B58F7702C086
:1053700084B58F7D84BD08958091B0008F7703C080
:105380008091B0008F7D8093B0000895CF93DF931C
:1053900090E0FC01ED50F44F2491FC01E95FF34FE4
:1053A0008491882349F190E0880F991FFC01E15D09
:1053B000F34FA591B4918B5D934FFC01C591D491AE
:1053C0009FB7611108C0F8948C91209582238C932B
:1053D000888182230AC0623051F4F8948C91322F74
:1053E000309583238C938881822B888304C0F89422
:1053F0008C91822B8C939FBFDF91CF910895A1E078
:10540000B0E0E5E0FAE20C94C02E282F30E0F9017C
:10541000E152F44F8491F901ED50F44F1491F901E8
:10542000E95FF34F04910023C9F0882321F06983D9
:105430000E949D296981E02FF0E0EE0FFF1FEB5DD8
:10544000F34FA591B4919FB7F8948C91611103C06B
:105450001095812301C0812B8C939FBF2196E4E09E
:105460000C94DC2ECF93DF93282F30E0F901E1522A
:10547000F44F8491F901ED50F44FD491F901E95FB3
:10548000F34FC491CC2391F081110E949D29EC2F00
:10549000F0E0EE0FFF1FE55EF34FA591B4912C9164
:1054A0002D2381E090E021F480E002C080E090E0D4
:1054B000DF91CF9108958E3008F08E508770209143
:1054C0009D0190E4299F90011124822B80937C0000
:1054D00080917A00806480937A0080917A0086FDC2
:1054E000FCCF809178002091790090E0922B089574
:1054F000A0E0B0E0EEE7FAE20C94BC2E6C017A0179
:10550000EB01E60EF71E00E010E0CE15DF0561F0BE
:105510006991D601ED91FC910190F081E02DC601D9
:105520000995080F191FF1CFC801CDB7DEB7E8E024
:105530000C94D82E6115710589F0DB010D900020C7
:10554000E9F7AD0141505109461B570BDC01ED91C4
:10555000FC910280F381E02D0995089580E090E0B0
:105560000895EF92FF920F931F93CF93DF938C01D7
:10557000FB01C0E0D0E064917F018FEFE81AF80AE8
:10558000662361F0D801ED91FC910190F081E02D4E
:10559000C8010995C80FD91FF701EDCFCE01CDB7CE
:1055A000DEB7E6E00C94DA2E0E949A2A0895DC0118
:1055B000ED91FC910190F081E02D099508950F93F4
:1055C0001F93CF93DF93EC016DE00E94D72A8C01EB
:1055D0006AE0CE010E94D72A800F911FDF91CF9100
:1055E0001F910F9108950F931F93CF93DF93EC01B9
:1055F0000E94B12A8C01CE010E94DF2A800F911FE8
:10560000DF91CF911F910F9108950F931F93CF9327
:10561000DF93EC010E949A2A8C01CE010E94DF2ABE
:10562000800F911FDF91CF911F910F9108950F93DC
:105630001F93CF93DF93EC010E94D72A8C01CE01F8
:105640000E94DF2A800F911FDF91CF911F910F9150
:105650000895A1E2B0E0EFE2FBE20C94B82E7C01E9
:10566000C42EE52FCB01D22E19A221E02D1510F06A
:105670002AE0D22E8E010F5D1F4F8D2C912CA12C74
:10568000B12C6C2D7E2FA50194010E94712E8C2DC2
:10569000D29E80191124015011098A3010F4805DC6
:1056A00001C0895CF8018083211531054105510550
:1056B00021F0C22EE32FCA01E4CFB801C7010E9436
:1056C0009A2AA196ECE00C94D42EA0E0B0E0EBE690
:1056D000FBE20C94BC2EEC016A017B012115310523
:1056E00041F4E881F9810190F081E02D642F099562
:1056F0001DC02A303105A9F477FF12C06DE20E9467
:10570000D72A8C0144275527BA014C195D096E0927
:105710007F092AE0CE010E94292B800F911F06C02D
:105720002AE0B701A601CE010E94292BCDB7DEB732
:10573000E8E00C94D82E9A01AB01662757FD6095DE
:10574000762F0E94652B08950F931F93CF93DF93BD
:10575000EC019A01AB01662757FD6095762F0E94F8
:10576000652B8C01CE010E94DF2A800F911FDF91F3
:10577000CF911F910F9108952115310549F4DC0156
:10578000ED91FC910190F081E02D642F0995089531
:105790000E94292B08959A01462F50E060E070E0A6
:1057A0000E94BC2B08959A01AB0160E070E00E945A
:1057B000BC2B08950F931F93CF93DF93EC010E94AE
:1057C000BC2B8C01CE010E94DF2A800F911FDF913C
:1057D000CF911F910F9108950F931F93CF93DF9354
:1057E000EC019A01AB0160E070E00E94BC2B8C01DF
:1057F000CE010E94DF2A800F911FDF91CF911F9170
:105800000F9108950F931F93CF93DF93EC019A01AB
:10581000462F50E060E070E00E94BC2B8C01CE016E
:105820000E94DF2A800F911FDF91CF911F910F916E
:105830000895FC0124853585F901E05CFF4F8081E6
:105840009181F901EE5BFF4F20813181821B930B27
:105850008F7399270895FC0184859585FC01E05C90
:10586000FF4F40815181FC01EE5BFF4F2081318170
:105870004217530741F00190F081E02DE80FF91F26
:10588000808190E008958FEF9FEF0895FC0184855B
:105890009585FC01E05CFF4F40815181FC01EE5B8E
:1058A000FF4F208131814217530779F0A081B181E8
:1058B000A80FB91F8C91208131812F5F3F4F2F732B
:1058C00033273183208390E008958FEF9FEF089571
:1058D000FC0181A1882329F0A489B5898C9186FFD8
:1058E000FBCF11A20895CF93DF93FC012685378566
:1058F000D901A05CBF4F8D919C91119701968F7338
:105900009927E901CE5BDF4F4881598184179507BC
:10591000D9F30D90BC91A02DA20FB31F6C93A68557
:10592000B785A05CBF4F11969C938E93A689B789CB
:105930002C9181E090E0078C02C0880F991F0A9497
:10594000E2F7282B2C9381E081A30488F589E02DD0
:1059500080818064808381E090E0DF91CF91089521
:1059600008951F920F920FB60F9211242F933F9319
:105970004F938F939F93EF93FF938091C00082FD8D
:105980001CC04091C60080918606909187060196C2
:105990008F73992720918806309189068217930783
:1059A00071F0E0918606F0918706EA5BF94F40833B
:1059B000909387068093860602C08091C600FF916F
:1059C000EF919F918F914F913F912F910F900FBE2B
:1059D0000F901F90189580EE95E00E94192C892B4E
:1059E00011F00E94B02C08951F920F920FB60F92E3
:1059F00011242F933F938F939F93EF93FF932091C5
:105A0000420630914306809144069091450628173E
:105A1000390731F48091C1008F7D8093C10014C09B
:105A2000E0914406F0914506EE5FF94F20818091A8
:105A300044069091450601968F73992790934506E9
:105A4000809344062093C600FF91EF919F918F9120
:105A50003F912F910F900FBE0F901F901895A0E0CF
:105A6000B0E0E5E3FDE20C94B82EFC011382128253
:105A700088EE93E0A0E0B0E084839583A683B783AB
:105A80008CEB93E091838083758764875787468783
:105A9000318B208B138B028BF58AE48AD78AC68AD6
:105AA000B18EA08E938E828E8F85848F8889858F0C
:105AB0008989868F8A89878F8B8980A3ECE00C94F3
:105AC000D42ECF92DF92EF92FF92CF93DF93EC012F
:105AD0006A017B01411581EE580761057105F9F0F6
:105AE000EC89FD8981E090E008A002C0880F991F31
:105AF0000A94E2F7808360E079E08DE390E0A7010B
:105B000096010E94712E2150310941095109569583
:105B1000479537952795211580E1380798F0EC894E
:105B2000FD89108260E874E88EE190E0A70196019B
:105B30000E94712E2150310941095109569547950E
:105B400037952795E889F9893083EA89FB8920838D
:105B500019A2EE89FF89408181E090E09C010C8CC4
:105B600002C0220F331F0A94E2F7422B4083EE89D2
:105B7000FF8940819C010D8C02C0220F331F0A94C3
:105B8000E2F7422B4083EE89FF8940819C010E8C15
:105B900002C0220F331F0A94E2F7422B4083EE89A2
:105BA000FF8920810F8C02C0880F991F0A94E2F7A9
:105BB000809582238083DF91CF91FF90EF90DF90DB
:105BC000CF9008958F929F92AF92BF92CF92DF9223
:105BD000EF92FF920F931F9381E08F9385E08F9355
:105BE00087E08F9383E08F9384E08F93E6EC8E2E93
:105BF000912CF2ECAF2EB12CA1ECCA2ED12CB0EC32
:105C0000EB2EF12C04EC10E025EC30E042E056E005
:105C100066E476E080EE95E00E942F2D0F900F90C5
:105C20000F900F900F901F910F91FF90EF90DF90CA
:105C3000CF90BF90AF909F908F9008950E9462295F
:105C40000E94A822CBEEDCE20E9454252097E1F3CB
:105C50000E94EB2CF9CFA29FB001B39FC001A39F7C
:105C6000700D811D1124911DB29F700D811D112495
:105C7000911D08950E942B2EA59F900DB49F900D0D
:105C8000A49F800D911D11240895B7FF0C943A2E06
:105C90000E943A2E821B930B0895DB018F939F93F2
:105CA0000E943A2EBF91AF91A29F800D911DA39F9C
:105CB000900DB29F900D1124089597FB072E16F4B6
:105CC000009407D077FD09D00E94EF2E07FC05D085
:105CD0003EF4909581959F4F0895709561957F4F03
:105CE0000895A1E21A2EAA1BBB1BFD010DC0AA1F1D
:105CF000BB1FEE1FFF1FA217B307E407F50720F035
:105D0000A21BB30BE40BF50B661F771F881F991FAF
:105D10001A9469F760957095809590959B01AC01F8
:105D2000BD01CF010895052E97FB1EF400940E943B
:105D3000AA2E57FD07D00E94712E07FC03D04EF407
:105D40000C94AA2E50954095309521953F4F4F4F7A
:105D50005F4F089590958095709561957F4F8F4F17
:105D60009F4F08952F923F924F925F926F927F9232
:105D70008F929F92AF92BF92CF92DF92EF92FF925B
:105D80000F931F93CF93DF93CDB7DEB7CA1BDB0B07
:105D90000FB6F894DEBF0FBECDBF09942A883988AC
:105DA00048885F846E847D848C849B84AA84B984B3
:105DB000C884DF80EE80FD800C811B81AA81B981BF
:105DC000CE0FD11D0FB6F894DEBF0FBECDBFED01D3
:105DD0000895EE0FFF1F0590F491E02D0994AA1B82
:105DE000BB1B51E107C0AA1FBB1FA617B70710F0C6
:105DF000A61BB70B881F991F5A95A9F780959095F8
:105E0000BC01CD0108958F929F92AF92BF92CF9225
:105E1000DF92EF92FF92CF93DF93EC01688179815B
:105E20008A819B81611571058105910521F464E2E8
:105E300079ED8BE597E02DE133EF41E050E00E94F2
:105E4000932E49015A019B01AC01A7EAB1E40E94DB
:105E50003A2E6B017C01ACEEB4EFA50194010E94D7
:105E6000482EC60ED71EE81EF91EF7FE06C081E0BA
:105E7000C81AD108E10880E8F80AC882D982EA8203
:105E8000FB82C701B6019F77DF91CF91FF90EF9022
:105E9000DF90CF90BF90AF909F908F9008950E9419
:105EA000032F089586E091E00E94032F08956093E8
:105EB00006017093070180930801909309010895EA
:105EC0002F923F925F926F927F928F929F92AF92AA
:105ED000BF92CF92DF92EF92FF920F931F93CF93D7
:105EE000DF938B01EA016115710521F0DB018C93D1
:105EF00011969C93209739F09E012250310923324C
:105F0000310508F0D8C07C016701BFEFCB1ADB0A6E
:105F10005601F7016080862D90E00E949230892B17
:105F200011F07601F1CFFDE26F120AC0570182E055
:105F3000A80EB11CD70111966C90772473940BC0F6
:105F4000BBE26B1207C05701E2E0AE0EB11CD701F5
:105F500011966C90712CCE018F7E892B89F4B0E361
:105F60006B1237C0F50180818F7D8835D1F4618057
:105F7000F2E0AF0EB11C872D8260782EC0E1D0E038
:105F8000CA30D10551F1C031D10521F0C830D10559
:105F900099F409C0CC24CA94DC2CEC2CAFE0FA2E86
:105FA00022C0209769F7C8E0D0E0CC24CA94DC2C4A
:105FB000EC2CFFE1FF2E17C06FEF7FEFCB019E01AE
:105FC000442737FD4095542F0E94712E69017A01B4
:105FD0000AC02097A9F6CAE0D0E0E9E9CE2EDC2C71
:105FE000EC2CE9E1FE2EF50160E020E030E0A901B3
:105FF0004E01AA2497FCA094BA2C1F0170ED572ED5
:10600000560CA9E0A51570F48FEB860D8A3118F4B3
:1060100099EC592E06C08FE9860D8A3148F589EA38
:10602000582E560C852D90E08C179D070CF56F3F70
:10603000D9F0C216D306E406F50698F0C501B401FE
:106040000E944D2E9B01AC01852D90E0A0E0B0E0B8
:10605000280F391F4A1F5B1F281739074A075B079C
:1060600010F46FEF01C061E03196D1016C90C5CFA3
:106070000115110551F0662311F0319703C071FE2F
:1060800004C03297D801ED93FC9370FE07C0509581
:106090004095309521953F4F4F4F5F4F67FF10C0A0
:1060A00082E290E090938B0680938A066FEF7FEFF9
:1060B0008FEF9FEF07C060E070E080E090E002C0EB
:1060C000B901CA01DF91CF911F910F91FF90EF901D
:1060D000DF90CF90BF90AF909F908F907F906F9008
:1060E0005F903F902F900895FC0188279927E894AE
:1060F00021912032E9F3293010F02E30C8F32B32F1
:1061000041F02D3239F4689404C00E94C630820FE9
:10611000911D219120532A30C0F31EF49095819552
:106120009F4F0895911150C0803219F089508550C9
:10613000D0F7089548EC53E00E949F300895FA018B
:10614000A191B081009719F41097E1F0CD01DC0125
:10615000CD010D90002011F4C00113C0FB0121916D
:10616000222319F02015D9F7F3CFFB012191201537
:1061700019F41E92119606C02223C1F70D9000203B
:10618000A1F7D001FA01A193B08308957AE0979F17
:10619000902D879F802D910D11240895F999FECFA0
:1061A00092BD81BDF89A992780B50895262FF99957
:1061B000FECF1FBA92BD81BD20BD0FB6F894FA9AEA
:1061C000F99A0FBE01960895992788270895F894A3
:0261D000FFCFFF
:1061D20000008C06200001000000FF000200020007
:1061E200020002000200020002000200020002009D
:1061F20002000200020002000200028025000005E7
:10620200400AA1204EA50020244EA52C2330C01206
:1062120000001A400AA1204EA5001B1E27522C2363
:10622200308025000005400AA1204EA50020244E02
:10623200A52C2330004B000006400AD0009D4900E7
:106242007B289D492C233000E1000005400A4501CE
:10625200D7DC03B81E0EBF00232E48E801008A4097
:106262000A6001555502AD1E20000023C801545892
:106272002074696D656F75742100596573004E6FE6
:10628200002C00386368004E2F41002C205B005D1B
:106292002028002900486F70206368616E6E656C6B
:1062A200200020402000456E746572696E6720618F
:1062B20064617074697665206368616E6E656C20D6
:1062C20073656C656374696F6E2C207069636B69AA
:1062D2006E673A007363616E6E6572206D6F6465FE
:1062E200004E4F5420454E41424C45440053656E8A
:1062F20064696E672073657474696E677320746F66
:106302002052580A00526573657474696E6720736F
:10631200657474696E6773206F6E2052580A00416B
:10632200626F727465642065646974730A00696ED1
:1063320076616C69642073656C656374696F6E0065
:106342000D0A496E76616C696420696E70757420FD
:106352002D2064697363617264656421070053656B
:106362007474696E677320736176656420746F203C
:10637200454550524F4D0A00526576657274656408
:106382002073657474696E67732066726F6D204541
:106392004550524F4D0A004C6F616465642066613E
:1063A20063746F72792064656661756C74730A0038
:1063B2004B657920616E64206368616E6E656C73F3
:1063C2002072616E646F6D697A65640A004F706550
:1063D2006E4C52536E672054582073746172746904
:1063E2006E672000206F6E20485720006D6F647525
:1063F2006C65206C6F636B65643F00342B3400382E
:1064020000382B340031320031322B340031360067
:1064120050504D0052535349005344410053434C92
:1064220000525844005458440041494E004C4245E1
:1064320045500053504B54524D0053425553005354
:10644200554D44004C4C494E440000070B0C1011B2
:106452001500B7012B032F033103350338033D0326
:10646200B7014003440349034D0351035503590344
:106472005D0363036A036F0374038D028D028D0251
:106482008D02160A1322312900000000732C782A8B
:08649200192C462C2B2C682C60
:00000001FF
